:1000000000000A128A110E28FE00030EF0000408F8
:10001000F1000A08F2000A168A15CE2D83010308A2
:08002000A0000A128A11C52F8D
:100034000F3083129000101080308F0000308E013A
:10004400101483160C140B17080082200A128A114C
:1000540003104A0D4B0DD1005108031D3628C5016C
:10006400C601C701C801080082200A128A1117308C
:100074000310CB0CCA0CC90CFF3E031D3A284908D7
:10008400CC00C617C7014508CD004608CE00470876
:10009400CF008E30D001D102D11F5D285108803AA3
:1000A4008F3E031C31280310D00CCF0CCE0CCD0C8A
:1000B400D10F55286B2818305102031831285108E4
:1000C40003196B280310CD0DCE0DCF0DD00DD10328
:1000D40061284C0803197928CD09CE09CF09D00924
:1000E400CD0A0319CE0A0319CF0A0319D00A5008FE
:1000F400C8004F08C7004E08C6004D08C5000800D8
:100104004508C9004608CA004708CB000800031088
:1001140003178312201E03140030031801308316C2
:100124000313EF0064001730831203178500F830BF
:100134008316031381000730031788000313850017
:10014400860103178901031387018312870186013E
:100154008501861285126430CF00D0010A168A11F7
:1001640026260A128A118B130A128A15D0270A121C
:100174008A110A128A111A200A128A110A128A1181
:10018400A7270A128A110A128A1504200A128A1150
:100194008B17F401F40AF5010A128A1570220A1267
:1001A4008A11750883160313CE007408CD0003303A
:1001B4000A128A157C220A128A1183160313DA00A2
:1001C40063308312C0009930C1006A30C2009A3093
:1001D400C300A0300A128A156F250A128A11A030B2
:1001E400CD000130CE000A128A155E250A128A114A
:1001F40083165A080319412991308312CD0099308E
:10020400CE000A128A155E250A128A110430F400FF
:10021400F5010A128A1570220A128A1175088316CA
:100224000313EE007408ED000630F400F5010A1221
:100234008A1570220A128A11750883160313D800CE
:100244007408D7001030F400F5010A128A157022E0
:100254000A128A11750883160313E0007408DF007C
:100264001E300A128A15A0220A128A11003A031DAE
:10027400412900300A128A15CA210A128A118312EE
:100284000317D730A201A3010313CD009A30CE0087
:100294000A128A15E7250A128A110A128A15B62744
:1002A4000A128A11031C83290A128A1174270A125A
:1002B4008A1183120317A300083A031D7429220824
:1002C40003198329A2032308F3000A128A1157276A
:1002D4000A128A112030F3000A128A1157270A12CF
:1002E4008A117A292208A03E840023088000A20AE9
:1002F400831203172308F3000A128A1157270A12DC
:100304008A11640083160313570858040319BF297C
:100314000A168A1100200A128A1173088312ED004A
:100324007408EE0083165808F4005708F3003C30B4
:10033400F500F6010A128A11A2260A128A1174081B
:100344006E02031DA72973086D02031CBF29C43064
:10035400CD009A30CE000A128A155E250A128A113F
:100364000A128A15AD260A128A1105308316EF0087
:1003740083120317A201A20AC9290D30831203179D
:1003840023060319C9291F302202031C4F292208FE
:100394009F3E8400A030831780010A128A158325AA
:1003A4000A128A1124080317A10003132308031750
:1003B400A00021080313EC00031720080313EB002B
:1003C4000A128A15CD220A128A114129A000F811B5
:1003D4000C18F815831603130C1083125F08831688
:1003E400A100A20183125E088316A300A401831254
:1003F4005D088316A500A60183125C088316A70076
:10040400A80183125B08FF3E8316A900FF3003187E
:100414000030AA002008643EAB000030031801300D
:10042400AC00831260088316B100A130B2013522FA
:100434000A128A114F088316C80083124E088316C5
:10044400C70083124D088316C60083124C08831616
:10045400C500F81D312A831603130C1408008316F3
:1004640003130C1008008312DA000A3E84001724D8
:100474000A128A11031D402A46305002031C502AD6
:10048400831203135A080A3E840017240A128A119D
:10049400031D4E2A8B305002031C582AFF3083124E
:1004A4000313D600D700D800D900CB2A8312031334
:1004B4005A08083E840083130008BE00840A00081A
:1004C400BF00BE0A0319BF0A5A080A3E8400000886
:1004D400BC00840A0008BD006C30BC070318BD0AC8
:1004E4000730BD075A08063E84000008C000840A8D
:1004F4000008C100D4220A128A113F08D9003E081C
:10050400D8003D08D7003C08D600B230BC00073004
:10051400BD00BE01BE0ABF01C001C00AC101D42290
:100524000A128A113C08D6023D08031C3D0FD7026B
:100534003E08031C3E0FD8023F08031C3F0FD9029C
:100544005A08043EFE231830A500A601A701A801FD
:100554000A168A117E270A128A1122240A128A1183
:100564005A08023EFE230A128A1139240A168A11F5
:100574007E270A128A1122240A128A115A08FE239B
:100584000A128A1139240A168A117E270A128A113C
:1005940022245908CF005808CE005708CD00560829
:1005A400CC0008003F08AB003E08AA0065230A12ED
:1005B4008A1140082A07C80041080318410A2B077A
:1005C400C9000030CA01CB013F02033003193E02C7
:1005D400031C142B3D08AF003C08AE003C230A1258
:1005E4008A112E082F04031DFA2A0230C600FC2AA1
:1005F400C601C60AC7014608C2004708C300003046
:10060400C31BFF30C400C5004208C8024308031CD2
:10061400430FC9024408031C440FCA024508031CC3
:10062400450FCB020130BC020030031CBD03BD02E8
:100634003D08AB003C08AA0085232A08C8072B08FC
:1006440003110318013E031DC9072C0803110318E5
:10065400013E031DCA072D0803110318013E031DA3
:10066400CB074B08BF004A08BE004908BD00480834
:10067400BC0008009030B001B00AAA000130AB0001
:100684002F08AD002E08AC000A128A117E260A1229
:100694008A112A082B040319612B2E080339031D20
:1006A400602B6430AA00AB012F08AD002E08AC000B
:1006B4000A128A117E262A082B040319B001300875
:1006C400AE00AF0108006430A300A4012B08F400BD
:1006D4002A08F300F130F5000B30F6000A128A11F3
:1006E400A2260A128A117308413EA5007408031851
:1006F400013EF43EA6000A128A1154262408AB00D7
:100704002308AA0008006430A300A4012B08A60053
:100714002A08A5000A128A1154260A128A112308EB
:10072400AE002408AF009030B001B101A300013045
:10073400A4002B08A6002A08A5000A128A11542630
:100744000A128A112308B2002408B300B401B501C7
:100754002B08B7002A08B6000310B70CB60C031018
:10076400B70CB60C3608B8003708B900BA01BB019B
:100774002A08A1002B08A2000130A301A401A801AA
:10078400A701A6006D30A5000A168A117E270A1259
:100794008A112108B80722080318220FB907230871
:1007A4000318230FBA0724080318240ABB073808C0
:1007B400B20739080318390FB3073A0803183A0F78
:1007C400B4073B0803183B0AB5072E08B2022F08EA
:1007D400031C2F0FB3023008031C300FB40231087E
:1007E400031C310FB5023508AD003408AC003308E2
:1007F400AB003208AA000800840083130008D0006C
:10080400840A0008D1005008D2005108D3000030F7
:10081400D31BFF30D400D5005908A4005808A30006
:100824005708A2005608A100080083130008D0004E
:10083400840A0008D100803AFF0080307F0208005B
:100844002108D20722080318220FD307230803180C
:10085400230FD40724080318240AD5075508D90000
:100864005408D8005308D7005208D60008003C307A
:10087400A500A601A701A8010800BF008312031365
:10088400E1260A168A1500200A128A11BE003E08C3
:100894000319432E25303E060319612C3F0A8400B8
:1008A4008313000803195D2CFA260A128A11002703
:1008B4000A128A11402CD5260A128A11402CBC0136
:1008C400BD01B5012F08FF002E0884000A168A1501
:1008D40000200A128A1146260A128A11031C492D85
:1008E400BC01BD010A30F300F4013D08F6003C08E8
:1008F400F500A2267408BD007308BC002F08FF0091
:100904002E0884000A168A1500200A128A11D03E85
:10091400B100FF3003180030B2003108BC070318DF
:10092400BD0A3208BD07AE0A0319AF0A2F08FF003B
:100934002E0884000A168A1500200A128A114626F7
:100944000A128A11031C492D742CBE260A128A111C
:10095400BA00840A00088403BB003A04031DB62CC1
:100964005C30BA009A30BB00B801B90138083A07C4
:1009740084003B0803183B0AFF000A168A1500206E
:100984000A128A11003A0319CB2CB80A0319B90ABE
:10099400B82C3D083902031DD12C3C083802031839
:1009A400DA2C3808BC023908031CBD03BD02DC2C58
:1009B400BC01BD01FF3083120313BC07031CBD033C
:1009C4003C0FE72C3D0A0319302D3F0A84008313A2
:1009D40000080319F42CF4260A128A1100270A12BB
:1009E4008A11DC2CC9260A128A11DC2C3F0A8400E5
:1009F400831300080319172D3B08FF003A088400ED
:100A04000A168A1500200A128A11F3003F0A84008C
:100A1400831300080A128A1100270A128A1183120A
:100A24000313BA0A0319BB0A302D3B08FF003A0826
:100A340084000A168A1500200A128A11B1003F08A0
:100A44008400831300088400310883178000BA0AE5
:100A54000319BB0A3F0884008313800A0130B802DB
:100A64000030031CB903B902380FF82C390A0319F2
:100A7400402CF82CBE260A128A11BE003E30BA0061
:100A8400BB01B801B80AB901CB2C3517632DE12697
:100A94000A168A1500200A128A11BE00003A0319A8
:100AA400432E633A03193C2D073A0319632D0D3A7B
:100AB4000319632D1A3A0319A72C063A0319472D73
:100AC400402D351B762DBE260A128A11B600840AE3
:100AD4000008B700B71F7D2D0330B504B609B70968
:100AE400B60A0319B70A7D2DBE260A128A11B6006A
:100AF400840A0008B700BE010530BE0A3E06031989
:100B0400992D03103E0DED260A168A1500200A12AF
:100B14008A11B1000A168A1500200A128A11B2003D
:100B24003702031D972D3108360203187E2D3C0829
:100B34003D040319A52D350803390319A52DFF30EC
:100B4400BC07031CBD033E08B100B201B11BB203D4
:100B54003208803AB3003D08803A3302031DB42DB5
:100B64003C0831020318C32D831203133E08B1005D
:100B7400B201B11BB203BC023208031CBD03BD02A7
:100B8400C72D83120313BC01BD013C083D040319A6
:100B9400E52D3F0A8400831300080319D82DF42699
:100BA4000A128A1100270A128A11DB2DC9260A1299
:100BB4008A11FF3083120313BC07031CBD033C08D6
:100BC4003D04031DCB2D350803390319052E3F0AB7
:100BD4008400831300080319FA2D2D30F3003F0A13
:100BE400840000080A128A1100270A128A11052EAD
:100BF4003F088400000884002D30831780003F08DC
:100C040084008313800A831203133E08B4003D2E2C
:100C14000A30AA00AB010310340DED260A168A151A
:100C240000200A128A11A3000A168A1500200A124B
:100C34008A11A4003708A6003608A50054260A1213
:100C44008A112408AD002308AC007E260A128A11FA
:100C54002A08303EBE003F0A8400831300080319AB
:100C64003A2EFA260A128A1100270A128A113D2EF8
:100C7400D5260A128A1183120313B403340F0A2EE1
:100C8400402CAE01AF010800F4003A30F3017402C5
:100C94000318522E30307402031C522EF301F30A4F
:100CA400730C0800A801A901230824040319792E50
:100CB400A701A70AA41B622E0310A30DA40D5B2E8B
:100CC4000310A80DA90D24082602031D6B2E23086A
:100CD4002502031C752E2308A5022408031CA60361
:100CE400A60228140310A40CA30CA70B622E290837
:100CF400A4002808A30008002A082B0403199D2E29
:100D0400F701F70AAB1B8A2E0310AA0DAB0D832E35
:100D14002B082D02031D902E2A082C02031C992E49
:100D24002A08AC022B08031CAD03AD020310AB0C64
:100D3400AA0CF70B8A2E2D08AB002C08AA00080079
:100D44008312A101A201731CAE2E75088312A107A0
:100D54000318A20A7608A2070310F50DF60D031076
:100D6400F40CF30C73087404031DA52E83122208DB
:100D7400F4002108F30008003008840083130008FD
:100D8400B1000230800731088400000808003F08E1
:100D94008400000884002030831780003F0884000A
:100DA4008313800A08003F088400000884003E087A
:100DB400831780003F0884008313800A08002F08EB
:100DC400B2002E08B100AE0A0319AF0A3208FF00C0
:100DD4003108840008001E3E840098300318013E48
:100DE400FF0008002030F3003F0A840000080800D8
:100DF4003E08F3003F0A840000080800FF000730A3
:100E04008A007F088207052F0A128A11572FA30030
:100E1400A4003D2F2308240603193D2F2030F3009E
:100E240057270A128A110830F30057270A128A1129
:100E34008312A4033D2F0830F30057270A128A11A6
:100E44002030F30057270A128A110830F30057277D
:100E54000A128A118312A4032408230203183D2FC3
:100E64001D2F24088400800123080800240884001E
:100E740021088000A40A6C270A128A118312A10097
:100E8400A2012208003A0319482F382F2108083AF2
:100E940003190C2F023A0319332F073A0319332F7E
:100EA400183A03192E2F382F0800831603135D08F0
:100EB400013E0F395E060319572F8B135D08103E50
:100EC4008400730883178000DD0A0F30DD050C16DB
:100ED4008B17080074270A128A11F400F3005727AD
:100EE400740808000A128A15B6270A128A11031810
:100EF4007D2F6400742F8B1383165B08903E84004F
:100F040083170008F300DB0A0F30DB058B17730827
:100F14000800063083166F0203189F2F03106F0D0D
:100F2400E13E8400831300088312CD00840A000884
:100F34008403CE000A128A155E2DE4308312CD009C
:100F44009A30CE000A128A155E2D193083160313C7
:100F540099001815181283129817181698128316E8
:100F64000C128C16181383121813831698129816E1
:0C0F74000B17DE01DD01DB01FA010800B3
:100F8A00C530F801F901FA0183138400E1300A122D
:100F9A008A150B200A128A11903083178400ED30CB
:100FAA000A128A150B200A128A1110308400203086
:100FBA000A128A150B2083169F30E1009A30E2004C
:100FCA009930E3009A30E400B530E5009A30E60043
:100FDA00B030E7009A30E800D630E9009A30EA00EB
:100FEA00DA30EB009A30EC003C30ED00EE01830180
:060FFA000A128A11892889
:10100800403083129F00803083169F0008006400E0
:101018008001840A04060319003404060C282830C9
:10102800CD009830CE005E25D401D501A830A300AC
:10103800A40183165F08FF3E8312A500831660088B
:101048000318013EFF3E8312A6000A128A11542695
:101058000A128A1555082402031D3428540823024D
:10106800031C6528540854075407D3002F30C000C8
:101078009930C1005508C3005408C2005308123EF5
:101088007C220A128A15643E0313C4000030031838
:101098000130C5005308133E7C220A128A15031337
:1010A800C600C7015308143E7C220A128A1503138E
:1010B800C800C90191220A128A15D40A0319D50A4F
:1010C8001A280C30F400F50170220A128A157508E6
:1010D8000313D0007408CF000830F400F501702223
:1010E8000A128A1575080313D2007408D100F0306B
:1010F800C0009830C100831660088312C3008316AD
:101108005F088312C20091220A128A156730C00054
:101118009830E4270A128A1591220A128A150E308D
:10112800F400F50170220A128A1575080313D0001D
:101138007408CF000A30F400F50170220A128A15EB
:1011480075080313D2007408D1009930C000983094
:10115800E4270A128A15912AA830A300A40183164D
:1011680060088312A60083165F088312A5000A127E
:101178008A1154260A128A152308E4002408E50077
:10118800640864076407E900123EE40000300318AD
:101198000130E500803AFF0080307F02031DD62829
:1011A800FE30640203180800A83083120313AA0053
:1011B800AB01831660088312AD0083165F088312A3
:1011C800AC000A128A117E260A128A152A082B04F4
:1011D800031D2929F4250A128A155F08E8005E080C
:1011E800E7009C30E7070318E80AFF30E8076808BB
:1011F800803AFF0081307F02031D04290030670216
:10120800031C0A29FF3083120313112983120313C5
:10121800E81F1029E60112296708E6006608F400AD
:101228006908123E55220A128A15F4018312031323
:101238006908133E55220A128A15F4018312031312
:101248006908143E55220A128A15790803190800FC
:10125800791C4B293A3083120313CD009A30CE0003
:101268005E250A128A150C30A100A201F400F501CE
:1012780070220A128A157408013E0313A300750828
:101288000318013E003EA40048220A128A15F91CE0
:101298006A294C3083120313CD009A30CE005E25A4
:1012A8000A128A150E30A100A201F400F50170227D
:1012B8000A128A157408013E0313A300750803185F
:1012C800013E003EA40048220A128A15791D892988
:1012D800433083120313CD009A30CE005E250A12E4
:1012E8008A150830A100A201F400F50170220A1243
:1012F8008A157408013E0313A30075080318013EFC
:10130800003EA40048220A128A15F91DA829543063
:1013180083120313CD009A30CE005E250A128A1577
:101328000A30A100A201F400F50170220A128A1500
:101338007408013E0313A30075080318013E003E1C
:10134800A40048220A128A157918AC29F91CBB296D
:10135800831203136908133E7C220A128A15013E80
:10136800F40003136908133E55220A128A158312E2
:1013780003136908143E7C220A128A15013EF40000
:1013880003136908143E5522F90108008312EA0084
:101398006A080319122AA530CD009A30CE005E25BE
:1013A8000A128A158316DF01E00183260A128A15BC
:1013B8000C30A100A201A301A40148220A128A1537
:1013C8000E3083120313A100A201A301A401482235
:1013D8000A128A15083083120313A100A201A3017F
:1013E800A40148220A128A150A3083120313A100A5
:1013F800A201A301A40148220A128A151230F4019D
:1014080055220A128A151330F40155220A128A1538
:101418001430F40155220A128A15192A7F30CD009A
:101428009A30CE005E250A128A1583160313DA0154
:10143800DA0A5A08F400033055220A168A11FC24E5
:101448000A128A15B0200A128A1583160313DF0AB6
:101458000319E00A10308312A100A2018316600864
:101468008312A40083165F088312A30048220A127D
:101478008A15AD260A128A150530A0220A128A1585
:10148800003A031D0800212A2408F40021085522E7
:101498000A128A15831203132308F4002108013E57
:1014A800552AF500831603178C18562A75088312D7
:1014B8008D0074088C003F3083168C0503108B1B3D
:1014C80003148B130C1555308D00AA308D008C1425
:1014D8000C1103188B1708007408013E7C220A12AD
:1014E8008A15F60074087C22F5007608F4000800D6
:1014F800F3006400831603178C187D2A730883127F
:101508008D003F3083168C050C1403100C1803143F
:101518000318013083120C0808000130CB01CC00FD
:101528004230CA004008AE004108AF004A30B0005F
:101538004B300A128A113F2C8312D400D630CD00CA
:101548009A30CE005E250A128A155408D50055082F
:1015580003190034BA30C0009A30C1005508C200DF
:10156800C30191220A128A15B6270A128A1503188E
:1015780001346400E83083120313CF000330D00035
:101588000A168A1126260A128A1583120313D5030E
:10159800AB2A6C08003A0319F22CED2CAD260A127E
:1015A8008A118B2F0A168A111828D030C0009A3059
:1015B800C10083166E088312C30083166D08831258
:1015C800C200A0306F250A128A15A030CD00013064
:1015D800CE005E2D0A128A118B2F0A168A15882DC5
:1015E800D030C0009A30C10083164C088312C30063
:1015F80083164B088312C200A0306F250A128A1581
:10160800A030CD000130CE005E2D0A168A11732855
:10161800D030C0009A30C100831658088312C30026
:10162800831657088312C200A0306F250A128A1544
:10163800A030CD000130CE005E2D86140030861813
:1016480001308316D900E2308312CD009A30CE00E3
:101658005E2D86100030861801308316D900E030E0
:101668008312CD009A30CE005E2DCC30C0009A3067
:10167800C100831659088312C200A030C3016F2528
:101688000A128A15A030CD000130CE005E2D0A1650
:101698008A11672CF4250A128A155F088316B4008C
:1016A80083125E088316B300F4255F088316B6001C
:1016B80083125E088316B5000A308312A300A401C2
:1016C800831634088312A600831633088312A500F4
:1016D8000A128A1154260A128A1524088316B80099
:1016E800831223088316B7000A308312AA00AB01BD
:1016F800831636088312AD00831635088312AC00B2
:101708000A128A117E260A128A152B088316BA0035
:1017180083122A088316B90071308312C0009A30E8
:10172800C100831638088312C30083163708831252
:10173800C20083163A088312C5008316390883123B
:10174800C400A0306F250A128A15A030CD000130E0
:10175800CE005E2D7430C0009A30C1004C300A169D
:101768008A11A5260A128A157708C3007608C200CE
:10177800A0306F250A128A15A030CD000130CE00A6
:101788005E2D7430C0009A30C10052300A168A119A
:10179800A5260A128A157708C3007608C200A03069
:1017A8006F250A128A15A030CD000130CE005E2DBB
:1017B8004C300A168A11E02852300A168A11E0289D
:1017C8000616E230CD009A30CE005E2D0612E030CB
:1017D800CD009A30CE005E2D8615E230CD009A30CD
:1017E800CE005E2D8611E030CD009A30CE005E2D01
:1017F8004C308E2F52308E2F0A168A11C72E0A1699
:101808008A11FC2C0A168A154B2DD130C0009A304B
:10181800C10000307C220A128A150313C200A030CE
:10182800C3016F250A128A15A030CD000130CE0001
:101838005E2DC830CD009A30CE00E7250A128A15F1
:10184800A030E3250A128A1583250A128A1523086F
:101858008316BF0012308312CD009A30CE00E725E0
:101868000A128A15A030E3250A128A1583250A125E
:101878008A1523088316C00008308312CD009A30D9
:10188800CE00E7250A128A15A030E3250A128A1528
:1018980083250A128A1523088316C1001C30831277
:1018A800CD009A30CE00E7250A128A15A030E3252C
:1018B8000A128A1583250A128A1523088316C2007C
:1018C80026308312CD009A30CE00E7250A128A15F9
:1018D800A030E3250A128A1583250A128A152308DF
:1018E8008316C30030308312CD009A30CE00E7252E
:1018F8000A128A15A030E3250A128A1583250A12CE
:101908008A1523088316C400FE308312CD0099304F
:10191800CE00E7250A128A15831640088312DB00D9
:10192800831641088312DC00831642088312DD0007
:10193800831643088312DE00831644088312DF00EF
:10194800A030E3250A128A1583252308E0008316B0
:101958003F080A128A11E829132883260A128A15D1
:1019680076088316BE007508BD007408BC007308AD
:10197800BB00BB3084270A128A15CD000130CE0087
:101988005E2D0130CA290030CA298316DA015A08A7
:10199800F400033055220A128A15BF30831203134C
:1019A800CD009A30CE005E2DD130C0009A30C100F3
:1019B800831660088312C30083165F088312C2006F
:1019C800A0306F250A128A15A030CD000130CE0054
:1019D8005E2D6A30CD009A30CE005E2D6B08013A3C
:1019E8000319D22A033A0319EE2A013A0319C52C1E
:1019F800073A0319C72C013A0319C92C033A0319EA
:101A0800D82C013A0319D62A0F3A0319D92A013AD0
:101A18000319F12A033A0319F42A013A0319092B85
:101A2800073A03190C2B013A03194B2B033A0319F4
:101A38004E2B013A0319062C1F3A0319092C013AB7
:101A480003191D2C033A0319B12C013A0319212B50
:101A5800073A03192D2B013A0319392B033A0319B5
:101A6800AE2B013A0319C52B0F3A0319DC2B013AA7
:101A78000319E02B033A0319E42B013A0319EA2B63
:101A8800073A0319F02B013A0319F62B033A031905
:101A9800FC2B013A0319FE2B3F3A0319002C013A9B
:101AA8000319002C033A0319032C063A0319B02C26
:101AB800ED2C08008630C0009A30C100D430C20036
:101AC8009A30C3004D08C4004E08C500D430C60083
:101AD8009A30C700912AC700C8004230C901C60021
:101AE8004008AE004108AF004630B00048300A1246
:101AF8008A113F24480884008317800108000313D3
:101B0800AA002A08840020300006031D8D2DAA0A89
:101B1800852D2A0884000930000603198B2DA80199
:101B2800A901A7012A0884002D300006031D9E2D57
:101B3800A70ACD2D2A0884002B3000060319CD2DC5
:101B48002A08840000080A128A1146260A128A15F1
:101B5800031CCF2D2A0884002908F4002808F30064
:101B68000A30F500F6010A128A11A2260A128A150D
:101B7800831700087307A5000030031801307407A5
:101B8800A6002508D03EA80026080318013EFF3EFF
:101B9800A900AA0AA42D27080319DE2D2809A500E3
:101BA8002909A600A50A0319A60A2508A3002608DC
:101BB800A40008002908A4002808A3000800F500CC
:101BC8000A128A11092F8830C0009A30C100D43017
:101BD800C2009A30C3004D08C4004E08C500912ABF
:101BE8000130831603178800031385008312061536
:101BF8006430CF00D0010A168A1126260A128A15E7
:101C080000300A168A11DB260A128A157408E100C8
:101C18007308E00006116108A5006008A400712699
:101C28000A128A152408B9002508BA002608BB003C
:101C380083164E088312A50083164D088312A4004C
:101C480071262408AA002508AB002608AC007A30C3
:101C5800A701A8004430A9000A168A151E260A12F0
:101C68008A152708B6002808B7002908B8000A16F8
:101C78008A1586260A128A153608C5003708C6004E
:101C88003808C7000A128A1127200A128A1546083E
:101C9800E3004508E2006308A5006208A400712675
:101CA8002408D5002508D6002608D7003F30D201E1
:101CB800D301D4000A168A15F3260A128A15520887
:101CC800C5005308C6005408C7000A128A11272005
:101CD8004608DF004508DE0008002408F300250850
:101CE800F4008E30F501F600F7010A168A15B327BD
:101CF8007308A4007408A5007508A60008007811E8
:101D0800831603130C187815831603130C10480850
:101D18008312A400831647088312A300831646087B
:101D28008312A200831645088312A100781DA02EF5
:101D3800831603130C14A32E831603130C1083129B
:101D48002408F6002308F5002208F4002108F3000F
:101D5800080083260A128A15EE270A128A15F72721
:101D68000A128A11A2260A128A157308D400740866
:101D7800D500D601D7015408D80755080311031810
:101D8800013E031DD907560803110318013E031D20
:101D9800DA07570803110318013E031DDB07C53096
:101DA800C0009930C10083166E088312C3008316E1
:101DB8006D088312C200A0306F250A128A15A03060
:101DC800CD000130CE005E250A128A15DC01DD0146
:101DD80083164C0883125D02031DF62E83164B08EA
:101DE80083125C0203180A2F6400E830831203137D
:101DF800CF000330D0000A168A1126260A128A1547
:101E080083120313DC0A0319DD0AEC2E8316981CCF
:101E18000A2F8C12831298138501860104308700DB
:101E28008316D9018312101080308F008E01101490
:101E380083160C140B178B13342F031E522F6300B9
:101E480083120313101080308F008E0110140C10B1
:101E58008316C50A0319C60A0319C70A0319C80A4B
:101E680083125D08D5005C08D400DC0A0319DD0A7A
:101E7800F7270A128A11A2260A128A157308FF3E4A
:101E8800D60074080318013EFF3ED70055085702D4
:101E9800031D502F540856020318212FD0270A1269
:101EA8008A158B17831D031E5B2F02305F2F831D3E
:101EB800031A602F0330EF0064308312CF00D00183
:101EC8000A168A1126260A128A150A128A11A727C3
:101ED8000A128A15DD308312CD009A30CE005E25B5
:101EE8000A128A1583260A128A15EE270A128A15FB
:101EF800583084270A128A15CD000130CE005E2D95
:101F08008312C2000A168A11D0200A128A150A16EC
:101F18008A11B02AD4004C3A031D942F0516952F28
:101F280085153230CF00D0010A168A1126260A12EA
:101F38008A154C30831203135406031DA52F05126E
:101F4800A62F8511AB30C0009A30C1005408C200DA
:101F5800A030C3016F250A128A15A030CD000130C8
:101F6800CE005E2D83120313981CC72F8316981278
:101F78009816831218121816C52F1A088316981265
:101F88009816031008001819C12F7A0883165B06E3
:101F98000319C52F031408007810831603130C18AF
:101FA8007814831603130C10C901CA01781CE02F9A
:101FB800831603130C140800831603130C1008006F
:101FC800C1005008C3004F08C2005208C50051089C
:101FD800C40008007608DB007508DA007408D90028
:101FE8007308D800080083166E08F4006D08F30023
:101FF8003C30F500F6010800F8100C18F8148316A8
:1020080003130C104A08F6004908F500F81C1028BC
:10201800831603130C141328831603130C10760865
:10202800F4007508F3000800D230CD009930CE00D6
:102038000A128A15E7250A168A11A0300A128A158B
:10204800E3250A168A11A0300A128A1583250A1672
:102058008A112408D0002308CF00500403196C28E3
:1020680004305002453003194F0203186C285008F9
:102078008316EE0083124F088316ED000430831296
:10208800A100A20183166E088312A40083166D08AE
:102098008312A3000A128A1548220A168A11CC3024
:1020A80083120313C0009A30C10083166E0883128E
:1020B800C30083166D088312C200A0300A128A1565
:1020C8006F25A030CD000130CE000A128A155E2D92
:1020D8006A30CD009A30CE000A128A155E2D4A3039
:1020E800CD009930CE000A128A15E7250A168A1102
:1020F800A0300A128A15E3250A168A11A0300A129E
:102108008A1583250A168A112408D0002308CF00CF
:1021180004305002453003194F020318C9285008EB
:102128008316D80083124F088316D700063083120F
:10213800A100A201831658088312A4008316570829
:102148008312A3000A128A1548220A168A11CC3073
:1021580083120313C0009A30C100831658088312F3
:10216800C300831657088312C200A0300A128A15CA
:102178006F250A168A11A030CD000130CE000A1250
:102188008A155E250A128A15D02F6A30CD009A303A
:10219800CE000A128A155E2DC10084008313000840
:1021A800BD00840A0008BE00840A0008BF00840A33
:1021B8000008C0003D301E29D6004C3A031DE62811
:1021C8000616E72886156330C0009A30C100560805
:1021D800C200A030C3010A128A156F250A168A1197
:1021E800A030CD000130CE000A128A155E250A16ED
:1021F8008A11D401D501003055021E30031954024A
:10220800031816296400E83083120313CF00033043
:10221800D00026260A168A1183120313D40A03193A
:10222800D50AFF284C305606031D1C290612080043
:1022380086110800B80084000008B900840A000864
:10224800BA00840A0008BB00840A0008BC003C30BD
:10225800CF270A168A1114220A168A112208831611
:102268000317DC0083120313210883160317DB000E
:102278003C30C0270A168A1109270A168A11E7274F
:102288000A168A113C30CF270A168A1114220A1618
:102298008A11220883160317DE008312031321080C
:1022A80083160317DD003C30C0270A168A11092758
:1022B8000A168A11E7270A168A111830CF270A1634
:1022C8008A1114220A168A11220883160317E000BD
:1022D80083120313210883160317DF001830C02761
:1022E8000A168A1109270A168A112A08831603175B
:1022F800E20083120313290883160317E10062081A
:10230800F6006108F5000430F5070318F60A0730EF
:10231800F300F401F1230A168A11740883160317CF
:10232800E8007308E7004630E500E601DC270A16F6
:102338008A117D220A168A11F8270A168A112F088F
:10234800803A3702031DAC292E0883160317610251
:10235800031CC62983160317DC270A168A117D2257
:102368000A168A112E0883160317E1028312031333
:102378002F0883160317031CE203E202E50A031978
:10238800E60A9A2983160317660883120313AF0017
:1023980083160317650883120313AE007D222E08E7
:1023A800B9000230B905831603176208EA0061080C
:1023B800E900E301E401831603176308123E840071
:1023C80098300318013E83120313FF000A168A157A
:1023D80000200A168A113904BA00F8270A168A1149
:1023E80080303702031DFC293A088316031761025F
:1023F800031C0E2A831203133A0883160317E102FB
:10240800031CE203E30A0319E40A8312031303100B
:10241800B90CDF2983160317E10A0319E20ADB3432
:10242800F401A81F242AA509A609A709A809A50A2D
:102438000319A60A0319A70A0319A80AF401F40A3A
:10244800A41F312AA109A209A309A409A10A0319F1
:10245800A20A0319A30A0319A40A240823042204BC
:1024680021040319662AF301F30AA41B412A031065
:10247800A10DA20DA30DA40D382A24082802031DBE
:102488004F2A23082702031D4F2A22082602031D6C
:102498004F2A21082502031C602A2108A5022208C8
:1024A800031C220FA6022308031C230FA7022408DB
:1024B800031C240FA8020310A40CA30CA20CA10C4B
:1024C800F30B412A74080319742AA509A609A70958
:1024D800A809A50A0319A60A0319A70A0319A80A2D
:1024E8002808A4002708A3002608A2002508A100A0
:1024F80008002E080339031DA62A6430AA00AB0180
:102508002F08AD002E08AC000A128A117E260A1682
:102518008A112A082B04031DAB2A9030AA00013027
:10252800AB002E082C3EAC002F080318013E013EDC
:10253800AD000A128A117E260A168A112A082B046F
:102548000319AB2A6D30AE000130AF0008006E30C1
:10255800AE000130AF00080083120313AC007B30DB
:10256800AA009930AB000330F3002C080C3E84001D
:10257800831700089E23AA070318AB0AA900A91B02
:10258800AB03C03083120313AD002B08FF002A08E9
:1025980084000A168A1500200A168A11B1270A161D
:1025A8008A1500200A168A11B1270A168A150020F2
:1025B8000A168A11A9002D088400290883178000AB
:1025C800AD0A2D08840020308000CB30AD0AAA0067
:1025D8009830AB000330F3002C08083E8400000854
:1025E8009E23AA070318AB0AA900A91BAB038312F1
:1025F80003132B08FF002A0884000A168A150020F6
:102608000A168A11B1270A168A1500200A168A1195
:10261800B1270A168A1500200A168A11A9002D0862
:102628008400290883178000203083160317C70009
:10263800831203132C08063E84000008A5002030EE
:10264800A600A700CA3077230A168A112C08043E70
:10265800F0270A168A11CD3077230A168A112C081A
:10266800023EF0270A168A11D03077230A168A11FB
:102678002C0884000008A5003030A6002030A700F0
:10268800D33077230A168A116430F300F4012C083A
:102698000A3E84000008F500840A0008F600AC230E
:1026A8000A168A117308133EA5002030A600D630FA
:1026B800A70177230A168A116430F300F4012C0865
:1026C8000A3E84000008F500840A0008F600F12399
:1026D8000A168A117308A5003030A6000A30A70030
:1026E800D8307723C034A8008400270883178000D7
:1026F800A803280884000A30F30025084B240A168A
:102708008A11303E80000A30F300250830240A166A
:102718008A11A50025080319982BA8032808840006
:102728002508303E80000800A803280884002608F1
:1027380080000800F500F40173087518F407031009
:10274800F30D0310F50C7508031DA02B7408080081
:10275800A201F41FB62BF309F409F30A0319F40ACA
:10276800A201A20AF61FBF2BF509F609F50A0319FB
:10277800F60A0130A206A301A40173087404031920
:10278800E42BA101A10AF41BCD2B0310F30DF40DCA
:10279800C62B0310A30DA40D74087602031DD62BB7
:1027A80073087502031CE02B7308F5027408031CF8
:1027B800F603F60223140310F40CF30CA10BCD2B33
:1027C80022080319EC2BA309A409A30A0319A40AD4
:1027D8002408F4002308F300080083120313A2015D
:1027E800F61FFD2BF509F609F50A0319F60AA201E9
:1027F800A20AF41F042CF309F409F30A0319F40AD2
:10280800730874040319232CA101A10AF41B102CCA
:102818000310F30DF40D092C74087602031D162C11
:1028280073087502031C1F2C7308F5027408031C37
:10283800F603F6020310F40CF30CA10B102C22087B
:1028480003192B2CF509F609F50A0319F60A760877
:10285800F4007508F3000800F400F6017308031982
:10286800492CF501F50AF31B3C2C0310F30D362C0B
:102878000310F60D73087402031C462C7308F40247
:1028880076140310F30CF50B3C2C76080800F500C1
:102898000830F600F7017508F40007300310F40C4F
:1028A800FF3E0310031D532C770D7404F70003102B
:1028B800F50D73087702031C632C7308F702F60BF7
:1028C8004F2C770808001130CD009930CE000A123D
:1028D8008A15E7250A168A11A0300A128A15E325F7
:1028E8000A168A11A0300A128A1583250A168A1137
:1028F8002408D7002308D60000305702C83003192F
:102908005602031CF52C01305702413003195602B8
:102918000318F52C0130831603178800031385006C
:10292800831206156430CF00D00126260A168A11B4
:102938000030DB260A168A117408D5007308D40003
:102948000611A9005508AA00AB01AC015608A10060
:102958005708A2000330A301A401A801A701A600FB
:10296800E830A5007E270A168A112408B00023083B
:10297800AF002208AE002108AD0009272A088316F7
:10298800CE00831229088316CD008312A101A10A63
:10299800A20183164E088312A40083164D088312E1
:1029A800A3000A128A1548220A168A11D030831207
:1029B8000313C0009A30C10083164E088312C30067
:1029C80083164D088312C200A0300A128A156F259B
:1029D8000A168A11A030CD000130CE000A128A15DD
:1029E8005E2D6A30CD009A30CE000A128A155E2D0F
:1029F8008312031306160530CF00D0012626831252
:102A080003138615EA30F901CD009930CE000A1279
:102A18008A155E250A168A11D401D501003055029F
:102A28001E30031954020318292D6400E83083125C
:102A38000313CF000330D00026260A168A1183120A
:102A48000313D40A0319D50A122D4C30A5260A16E9
:102A58008A1177088316D0007608CF00013050021B
:102A68002C3003194F02031C791464308312CF00F1
:102A7800D00126260A168A115230A5267708831611
:102A8800D4007608D300013054022C3003195302C5
:102A9800031C7915DE308312C0009930C1008316FB
:102AA80050088312C30083164F088312C20083168E
:102AB80054088312C500831653088312C400A0303B
:102AC8000A128A156F250A168A11A030CD00013026
:102AD800CE000A128A155E250A168A118D30CD009D
:102AE8009A30CE000A128A155E250A168A118614B3
:102AF8000030861801308316D9008312D401D5011D
:102B08006400E83083120313CF000330D000262678
:102B18000A168A1183120313D40A0319D50A00303E
:102B28005502073003195402031C842D7830C00065
:102B38009A30C100831660088312C30083165F08A9
:102B48008312C200A0300A128A156F250A168A114C
:102B5800A030CD000130CE000A128A155E250A1673
:102B68008A11C7260A168A11D401D5016400E830F3
:102B780083120313CF000330D00026260A168A11C9
:102B880083120313D40A0319D50A003055020A30F8
:102B980003195402031CBA2D9330CD009A30CE008D
:102BA8000A128A155E250A168A11861106128610DF
:102BB8000030861801308316D9004C30A5260A1635
:102BC8008A1177088316D2007608D10000305202A5
:102BD8006530031951020318F91464308312CF00C9
:102BE800D00126260A168A115230A52677088316A0
:102BF800D6007608D5000030560265300319550214
:102C08000318F915DE308312C0009930C10083160D
:102C180052088312C300831651088312C200831618
:102C280056088312C500831655088312C400A030C5
:102C38000A128A156F25A030CD000130CE000A1285
:102C48008A155E2D812E0730D2007D30D100D10B40
:102C58002B2ED20B2B2E08002130D2007630D1003B
:102C6800D10B342ED20B342E000008004130D20094
:102C7800EE30D100D10B3E2ED20B3E2E00000800C4
:102C88008230D200DD30D100D10B482ED20B482E35
:102C98004D2E08000230D3008630D2009930D10082
:102CA800D10B542ED20B542ED30B542E08000630C1
:102CB800D3001330D200B130D100D10B612ED20B2A
:102CC800612ED30B612E682E0800B630C0009930F3
:102CD800C1005008C3004F08C200A0300A128A156C
:102CE8006F250A168A11A030CD000130CE000A12D5
:102CF8008A155E250A168A11442E5008003A0319CF
:102D08008C2E013A03199A2E023A03199F2E692E26
:102D18004F08053A0319272E1C3A0319302E2B3A6F
:102D280003193A2E563A0319442E692E4F082C3AA5
:102D380003194E2E692E4F08E83A03195B2E692EA7
:102D4800080083120313A6000730831603178800B0
:102D5800031385004C30831226060319B52E023062
:102D6800B62E0130DB267408A8007308A7002808CF
:102D7800A5002708A4000310A50CA40C2408F6003D
:102D88002508F700080085163230CF00D001262626
:102D98000A168A118312031386162C30CF000130CD
:102DA800D000262683120313861285120800831288
:102DB8000313A1000F30A105C3309F052108F500BA
:102DC80001300310F50DFF3E0310031DE62E750DAF
:102DD8009F041F14F930F5000000F50BF02EF42EB7
:102DE8000000831203139F149F18F82E1E08A300D7
:102DF800A20183161E088312A2070318A30A1F1034
:102E08002308F4002208F3000800B201AC1F192FB0
:102E1800A909AA09AB09AC09A90A0319AA0A03193D
:102E2800AB0A0319AC0AB201B20AB01F282FAD09C8
:102E3800AE09AF09B009AD0A0319AE0A0319AF0A02
:102E48000319B00A0130B206B301B401B501B601E5
:102E58002C082B042A0429040319672FB101B10A8D
:102E6800AC1B3C2F0310A90DAA0DAB0DAC0D332FD5
:102E78000310B30DB40DB50DB60D2C083002031DAB
:102E88004F2F2B082F02031D4F2F2A082E02031D38
:102E98004F2F29082D02031C612F2908AD022A088B
:102EA800031C2A0FAE022B08031C2B0FAF022C08A1
:102EB800031C2C0FB00233140310AC0CAB0CAA0C7F
:102EC800A90CB10B3C2F32080319752FB309B409AB
:102ED800B509B609B30A0319B40A0319B50A0319DF
:102EE800B60A3608AC003508AB003408AA00330827
:102EF800A9000800F301F401F501F601211C982F3F
:102F08002508F307260803110318013E031DF407DB
:102F1800270803110318013E031DF50728080311AC
:102F28000318013E031DF6070310A50DA60DA70DF6
:102F3800A80D0310A40CA30CA20CA10C24082304B4
:102F480022042104031D822F7608A4007508A3001B
:102F58007408A2007308A1000800A9002D088400C5
:102F6800290883178000AA0A0319AB0AAD0A2B089F
:102F7800FF002A088400080083120313A900AA018D
:102F8800AB01AC013C08B0003B08AF003A08AE000A
:102F98003908AD000800A100A201A301A4013C0862
:102FA800A8003B08A7003A08A6003908A5000800B1
:102FB800660883120313AF0083160317650883128C
:102FC8000313AE0008002C08BC002B08BB002A081D
:102FD800BA002908B900080084000008A5003030AC
:102FE800A6003A30A7000800831603176208803A43
:102FF80083120313B7000800FF1B0A2883137F18E6
:1030080083170008840A0319FF0A08007F087F391C
:103018008A000408840A0319FF0A82001F341C343A
:103028001F341E341F341E341F341F341E341F3403
:103038001E341F34013400340A340034643400343C
:10304800E8340334103427345734653465346B342A
:1030580020344E346F342E342C34203456346F34AC
:103068006C3474346134673465342034283456340D
:1030780029342C3420344C34653466347434203488
:103088005334743472346F346234653420344634C3
:10309800613475346C34743473342C3420345234C1
:1030A8006934673468347434203453347434723473
:1030B8006F346234653420344634613475346C348A
:1030C8007434733400340D3420344C34653466342D
:1030D8007434203455346E346434653472342D3489
:1030E8004334683461347234673465343A34203494
:1030F80025343334643409345234693467346834D9
:103108007434203455346E346434653472342D3458
:103118004334683461347234673465343A34203463
:103128002534333464340A3400340D3420344C34B8
:10313800653466347434203420344F34763465343E
:1031480072342D34633468346134723467346534CE
:103158003A342034253433346434093452346934ED
:10316800673468347434203420344F34763465340A
:1031780072342D34433468346134723467346534BE
:103188003A3420342534333464340A3400344A342D
:1031980061346E344634653462344D34613472348B
:1031A8004134703472344D34613479344A3475346E
:1031B8006E344A3475346C3441347534673453345E
:1031C800653470344F34633474344E346F34763429
:1031D80044346534633400340A340D3454344F3481
:1031E800543441344C3420344634413455344C340E
:1031F8005434533420344F345534543420344F34F9
:103208004634203425346434203449344D34413430
:103218004734453453340A34003444346534633411
:10322800693476346F346C347434733428343234FB
:10323800303430342D343334323430342C34303468
:103248003D343D34613462346F347234743429341B
:103258003A34203400340D342034203420342534DA
:10326800323464342C340934093425343334643426
:103278002C34093409342534333464342C34093477
:1032880009342534333464340A34003431342D3469
:10329800313430343934323420346D3469346E3456
:1032A8002C3430343D343D3466346F3472346534F4
:1032B80076346534723429343A342034003457343F
:1032C80061346B34653479342034253473342034D4
:1032D800433461346D346534723461342034543489
:1032E8007234693470346F346434213400345334A4
:1032F80075346E344D346F346E34543475346534EB
:10330800573465346434543468347534463472340C
:10331800693453346134743400344134633474345C
:1033280069347634653420344434653470346C340C
:103338006F3479346D3465346E3474342134003428
:1033480031342D343234353435342C34303420345F
:1033580074346F342034613462346F3472347434AA
:103368003A3400344E346F342034643465346C3469
:103378006134793420342534643420346D34733422
:10338800003453346C346534653470342034253457
:10339800643420346D3469346E34003431342D345F
:1033A800313430343934323420346D3469346E3445
:1033B8003A3400344C343A34253475345634203495
:1033C80052343A342534753456340034433468342E
:1033D80061347234673465342E342E342E3400341C
:1033E80030342D3436343034203473346534633417
:1033F8003A340034443453345434283430342D347B
:10340800313429343E34003444344434283431349B
:103418002D343334313429343E3400344D344D3472
:10342800283431342D343134323429343E340034A4
:1034380048344834283430342D3432343334293441
:103448003E3400344D344D34283430342D34353442
:10345800393429343E340034533453342834303426
:103468002D343534393429343E3400344C34533413
:10347800203475346E346434653472340034523414
:103488005334203475346E34643465347234003403
:103498004C34533420346F34763465347234003409
:1034A8005234533420346F347634653472340034F3
:1034B80028346E3475346C346C3429340034253433
:1034C800633420342E342E342E34003476343134A0
:1034D8002E3434342E3433340034253475342E34B9
:1034E800253475345634003449346D346734203407
:1034F80025346434003452346534733475346D348F
:1035080065340034253473342534733425347334E6
:103518000034433461346D3473342B340034433411
:1035280061346D3473342D3400345234533454348C
:103538005734443400345234533454344F344B34B5
:10354800003442346534673469346E3400342534C9
:10355800633420342134003457344B3457344434E2
:10356800003457344B344F344B3400340D34253445
:10357800333464340034483461346C347434003483
:1035880054344F3421340034593459343E340034DF
:103598003D342534643400343D34253475340034E6
:1035A8000D340A3400343E342034003454344F345B
:1035B800003455347034003430340034313400343D
:0435C8003F34003458
:103A9600A430CD009930CE000A128A15E7250A1601
:103AA6008A15A0300A128A15E3250A168A15A0304F
:103AB6000A128A1583250A168A152308CF004F088D
:103AC6000319812D4F08F40000300A128A15552279
:103AD6000A168A15D03083120313C0009A30C1002B
:103AE6004F08C200A030C3010A128A156F25A03004
:103AF600CD000130CE000A128A155E2D6A30CD0047
:103B06009A30CE000A128A155E2DF430CD00993017
:103B1600CE000A128A15E7250A168A15A0300A125F
:103B26008A15E3250A168A15A0300A128A158325F6
:103B36000A168A152408D0002308CF000030500248
:103B46003D3003194F020318C72D50088316CC00C9
:103B560083124F088316CB00CC308312C0009A30F4
:103B6600C10083164C088312C30083164B088312C8
:103B7600C200A0300A128A156F25A030CD00013090
:103B8600CE000A128A155E2D6A30CD009A30CE001C
:103B96000A128A155E2D831203138C1EE82D8316D6
:103BA6008C1EE82D7A08903E840083121A0883172B
:103BB60080007A08013E8316DC000F30DC055C08C5
:103BC6005B060319E82D5C08FA0083120C1EFD2D16
:103BD60083160C1EFD2D5E08103E84008317000818
:103BE600831299008316DE0A0F30DE055E085D0635
:103BF60003190C1283160C1C152E83120C1C152E81
:103C0600101080308F008E0110148316C90A031914
:103C1600CA0AC50A0319C60A0319C70A0319C80A34
:103C260083120C1072088A0071088400700E8300DB
:103C3600FE0E7E0E09002A08AD002B08AE002C08E9
:103C4600AF0003102E0D2F0DB4003408031D2F2EC8
:103C5600A701A801A90108002708AD002808AE00A1
:103C66002908AF0003102E0D2F0DB5003508031DD2
:103C7600402EA701A801A90108008930B101B201AF
:103C8600B3013507AD00B4022C08B5002908B50606
:103C96008030B5051830AB17AC01A817A901B000E4
:103CA6000310B10DB20DB30D29082C02031D612EB0
:103CB60028082B02031D612E27082A02031C6F2EDB
:103CC6002708AA022808031C280FAB022908031C90
:103CD600290AAC0231140310AA0DAB0DAC0DB00BC2
:103CE600532E3108F3003208F4003308F500340887
:103CF600F6003508F700B3277308A7007408A80074
:103D06007508A90008003608BC003708BD00380849
:103D1600BE0003103D0D3E0DBF003F08031D972E4C
:103D2600B601B701B80108003908BC003A08BD0061
:103D36003B08BE0003103D0D3E0DC4004408031DA4
:103D4600A82EB601B701B801080044087B3EBF079C
:103D56003808C4003B08C4068030C4050730B717CE
:103D6600BA17BB01C001C101C201C300361CC22E75
:103D7600F5270A168A1503183B0A031DC207031006
:103D8600B80CB70CB60C0310B90DBA0DBB0DC30BAE
:103D9600B92E0930C300361CD72EF5270A168A1508
:103DA60003183B0A031DC2070310B80CB70CB60C68
:103DB6000310C20CC10CC00CC30BCE2E4008F3007E
:103DC6004108F4004208F5003F08F6004408F700F1
:103DD600B3277308B6007408B7007508B800080062
:103DE6005208D8005308D9005408DA000310590DB8
:103DF6005A0DDD005508D8005608D9005708DA00D4
:103E06000310590D5A0DDC005D080319162F5C08C6
:103E16005D025C0803181E2FD8005D08D802193011
:103E26005802031C1D2F5508D2005608D300570808
:103E3600D40008005C08031908005D085C0203183A
:103E46002C2F5D08D8005C08D802193058020318D8
:103E560008000630DB00D41BDB17D71B5B17D31714
:103E6600D401D617D7015C085D020318532F03103F
:103E7600D50DD60DD70DDC035C085D0603194E2F54
:103E8600DB035B08073903194E2F3A2F0310D40CB6
:103E9600D30CD20CDD0A5D085C0603196F2F492F7F
:103EA6005D085C0203186F2F0310D20DD30DD40DDD
:103EB600DD035C085D0603196B2FDB035B0807391E
:103EC60003196B2F572F0310D70CD60CD50CDC0A11
:103ED6005D085C06031D662FDB1F7A2FFF30D206B6
:103EE600D306D406D20A0319D30A0319D40A5B1FD0
:103EF600852FFF30D506D606D706D50A0319D60A6A
:103F06000319D70ADB015208D50753080311031812
:103F1600530A031DD607540803110318540A031D38
:103F2600D707D71FA12FFF30D506D606D706D50A45
:103F36000319D60A0319D70ADB01DB0A5508F30071
:103F46005608F4005708F5005D08F6005B08F70010
:103F5600B3277308D2007408D3007508D40008008C
:103F660076080319BB2F750874047304031DC42F48
:103F7600F301F401F5010800F60A0310F50CF40C40
:103F8600F30CFE3075050319D32FBF2FF60AF30A7B
:103F96000319F40A0319F50A0310F50CF40CF30CD3
:103FA600FF3075050319E12FC92F02307602031C75
:103FB600E32FF6030310F30DF40DF50DF41FD82FC0
:103FC600761CF4130310F60C7608A300A201A101D7
:103FD6002108F3042208F4042308F5047708031DD6
:103FE600F51708003908C0073A08031103183A0AFA
:0A3FF600031DC1073B08031108007A
:02400E00DAECEA
:00000001FF
